:040000006F10B007C6
:1000040000000000000000008015000082150000C0
:10001400000000007818000000000000000000004C
:1000240078180000781800000000000000000000AC
:100034008415000000000000781800000000000093
:10004400781800007818000078180000781800006C
:10005400781800007818000078180000781800005C
:10006400781800007818000078180000781800004C
:10007400781800007818000078180000781800003C
:10008400781800007818000078180000781800002C
:10009400781800007818000078180000781800001C
:1000A400781800007818000078180000781800000C
:1000B40078180000781800007818000078180000FC
:1000C40078180000781800007818000078180000EC
:1000D40078180000781800007818000078180000DC
:1000E400E015000078180000781800007818000067
:0C00F40078180000781800007818000050
:10010000397101436EC619A0397141536AC866CA74
:1001100062CC5ECE19A0397101535AD056D252D456
:100120004ED64AD826DA22DC06DE330161408282CE
:1001300041114AC026C222C406C68282B24D410184
:10014000024D924C224CB24B4101024B924A224A40
:10015000B2494101024992442244B24041018280A5
:100160003D432A876373C3029377F700BDEFADE584
:10017000937606FF3D8ABA960CC34CC30CC74CC796
:100180004107E36BD7FE11E28280B306C3408A06C3
:100190009702000096966780A6002307B700A30683
:1001A000B7002306B700A305B7002305B700A304D3
:1001B000B7002304B700A303B7002303B700A302CB
:1001C000B7002302B700A301B7002301B700A300C3
:1001D000B7002300B700828093F5F50F9396850052
:1001E000D58D93960501D58D61B79396270097021B
:1001F000000096968682E78086FA9680C1171D8F4A
:100200003E96E374C3F8A5B7EFF29FF22E869305EE
:10021000100AEF0020783DBFEFF29FF1B7170140C1
:10022000214798CB2E89B2849305000A1306E00A71
:100230002A84EF0020764A8622859305000AEF0083
:100240006075A6852285C93731B711CEEFF25FEE12
:10025000C1479376F60F63F3C700C1462E86930518
:100260000009CD2BC5BD8280EFF29FEC91E1854561
:100270009205C51593F5F50FF12BE9BDEFF25FEB94
:1002800001111306000281450A85D93D1165EF1061
:10029000B0583724014013050440EF106066B707DB
:1002A0000E003EC68A85854713050440230AF100E7
:1002B00002C002C202C402C8EF10E0689D460546B3
:1002C000130504408D45EF10E06F8545130504408C
:1002D000EF10C06C0561BDBDEFF29FE53725014011
:1002E000854513050540EF10606CADB5EFF25FE496
:1002F0000564B72401407D141389044089454A856B
:10030000EF10407819E511E0B1B57D144204418049
:10031000F5B77DD813850440EF1040762399A1806E
:10032000E5B72388A1809307F00F6315F502EFF27C
:100330003FE0B7050020938705003147371501409E
:100340009AA39385050041471305058098C7EF10D0
:10035000102309B5828003C501818280EFF2BFDBE3
:10036000938401819C209306F00F638ED70085490A
:10037000638B370791CB1384018109476381E708B9
:100380000D476383E70ED1B337140140B147232AE9
:10039000F480370A002023803401A14A23285481A5
:1003A00013090A001304048091472310F9009305F0
:1003B0000A009307800222852324F900EF10301CE5
:1003C00093050A0022852310590123240900EF1008
:1003D000101B1937B707002003C707062380340115
:1003E000238AE1804DB783C741811384418181E72E
:1003F000E53589479CA01C20FD171CA069B7FD3579
:10040000B7050020938705003147371501409AA3AF
:100410009385050041471305058098C7EF103016F6
:1004200003D7218193060069B70700209387070649
:1004300063F4E60298239306F00305071377F70F9A
:1004400063E4E60098A311A094A39C2393C7F7FF4D
:10045000238AF1808D4755B79306F059E3E7E6FE0E
:10046000982365D77D17F9BF03C7418193874181E1
:1004700019E3238004007D1798A331B7B707002044
:1004800003C50706828001E903D721819307F0188D
:1004900063E7E70082809307F00263E8A7008967BB
:1004A000938787443E950821828019458280EFF228
:1004B0003FC8EF00907693878185114798A3D8AB0A
:1004C00051B9EFF25FC5C169138481858144914AB6
:1004D000FD19114B054A034904002685137989004B
:1004E000EF00306A3DCD3E206384370185073EA092
:1004F0003A206371EB061C2093F617008DE2936798
:1005000019001CA01C44B9C76316090426858297EC
:100510001C2093E707011CA035A885446DBF562019
:10052000636AD70213F7270019C37A2005C793E738
:1005300027001CA05C4489CB63180900268582979C
:100540001C2093E707021CA07A203E2063F8E700F6
:10055000231104005104E39244FDC5BE998F3EA0CF
:10056000D5BF1C20918BFDF71C482300540123119B
:100570000400EDD3E31009FE268582971C2093E743
:10058000070451BFEFF2DFBAEF1060501317850078
:10059000B7060200634307029357050193F7F70F6D
:1005A0009387D7FC1947C1666369F7000547B317FE
:1005B000F70093F7970791C3A166368561BEEFF206
:1005C0009FB537090008B7E9242021448144130A64
:1005D000F00F13090980938929C37D141374F40F54
:1005E00063194407C5E49387018823A00188138712
:1005F00007021385018823820700A3820700238353
:100600000700A38307009107E317F7FE9967938715
:1006100007485EA19307001C5EA589477CB58567E6
:10062000938707C85EA9AD477CB901478147930608
:1006300060033306E50010220507B297C207C183A5
:10064000E319D7FE7EB9B7E72420938727C31CDDC3
:10065000EDBC0D3F93178400CA973E951C5DE39E49
:1006600037F77639130665032A8781470C23050778
:10067000AE97C207C183E31BE6FEE390F6F61C418A
:10068000E3FDF4F4A38A8180BE8481BFE53D83C588
:100690005181B707000893870780A205BE95AA95E8
:1006A0001306C00313850188EF10F04E55B7EFF223
:1006B0003FA8138701881C439386018813066003B3
:1006C00085071CC301478147B385E6008C210507D8
:1006D000AE97C207C183E319C7FEFEBAB7E724206D
:1006E000938727C39CDE93875181802305041D884F
:1006F00080A3493DB70700089387078022043E94F2
:100700009385018822951120B1B4EFF27FA22E8942
:1007100093050010AA84EF10204291472A846306B3
:10072000F5009377F50F3E8535B413060010CA85A2
:100730002685EF10E0578147E30785FE9377F50F95
:10074000DDB789E590A310A390A28280135885405D
:100750001378F80F954863EC0803937828006385B5
:100760000800B688BE86C68793784800638508006F
:10077000BA883E87C6871373180013786800631A17
:100780000800631A03003688BA86428729A01548F4
:10079000E1BFE31A03FE10A313C8F5FF1317060108
:1007A00041831378F80F33080703C205C18105821E
:1007B00005084208135808019358880046984208D3
:1007C000135808011358880023800701631003049D
:1007D0001375F50F0DE5A20593D78500BE95939788
:1007E0000501C183A18393C7F7FF93F7F70FB30701
:1007F000F702B297C207C183A1839CA2828033050E
:10080000A0401375F50FB385A502F9B71375F50F61
:10081000DDBFEFF2FF91B7370A0041119387A7C2FE
:10082000375400403EC0B707000411679387F707AD
:1008300002C202C68A851305044078833EC47886C6
:10084000EF100063854513050440EF10E07141018E
:100850006FF05F90EFF23F8CFD77FD173759004046
:10086000239BF1802A8BAE8AB284B689138461817E
:1008700013090940B70502004A85EF10607611C5DB
:100880001E201387F7FF1AA0F5F71E207D55E5C33C
:1008900037590040130509408545EF10606EFD771C
:1008A000FD17370A03001EA0050A13090940D28567
:1008B0004A85EF10807111E51E201387F7FF1AA0FB
:1008C000FDF71E207955C5C737590040130509406B
:1008D0000146DA85EF10406EFD77FD17370A0700F5
:1008E0001EA0130A2A0813090940D2854A85EF1071
:1008F000C06D11E51E201387F7FF1AA0FDF71E201B
:100900007555B5C73759004013050940D685EF1016
:10091000606AFD77FD17370A07001EA0130A4A0810
:1009200013090940D2854A85EF10206A11E51E207F
:100930001387F7FF1AA0FDF71E2071558DCB375492
:1009400000403709001013040440370A0700A69935
:1009500013090908A28A130A4A08639C340137550F
:100960000040130505408545EF10206301456FF0F9
:10097000CFFDCA852285EF10A06665D1850483C5A9
:10098000F4FF5685EF100063D2852285EF10E063F7
:1009900065DDE1B7EFF2CFF94111D0878546130647
:1009A000F1004D3D41016FF0EFFAEFF26FF80111E8
:1009B00002C202C42316010002C802CA02CC02CE3F
:1009C00081471387C18B930600043306F700230089
:1009D00006008507E39BD7FE9387C181239007001C
:1009E0003D46930510051305800623810700EFF0AF
:1009F000BF82896541469385854713058006EFF0E0
:100A0000DF84370400409307F03F4C001305044097
:100A10003EC402C2EF10E072C167938707063EC86A
:100A20000C08894713050440FC84231B0100EF10C8
:100A3000E0770C0813050440EF10E07D0C08130567
:100A40000440EF10B006130504408545EF10D010A8
:100A5000130504408145EF1030131305044085450C
:100A6000EF10F010854513050440EF10700D05617F
:100A70006FF04FEE0547238CE180828003C78181B0
:100A800041C7EFF2EFEA3971138481811387C18B7B
:100A90008A8613054702B6859387C18B368603C8BD
:100AA000070091078505A38F05FF03C8D7FFA3871C
:100AB000050103C8E7FFA38F050103C8F7FFA3875C
:100AC0000503E39EA7FC9307C7018345470211076F
:100AD000FD168CAA834517022380B60283452702A0
:100AE0002388B602834537022380B604E31FF7FC50
:100AF00093060004854513058006EFF0EFF623000A
:100B0000040021616FF00FE58280EFF26FE2411186
:100B1000EFF0DF96EFF03F97340001471386C18175
:100B20000D488D45B307E6009C2305078906B307EA
:100B3000F502C207C1839983B38707038583239F87
:100B4000F6FEE311B7FE370400401305044081456B
:100B5000EF109000188689679387874806073E97AD
:100B60001A231305044085455AB9188506073E9790
:100B70001A231ABD18840607BA979E235EBDEF108C
:100B8000A07D41016FF00FDDEFF28FDA1386C18295
:100B90001C2205476380E7081384C18289CB09477B
:100BA0006387E7000D476385E70A6FF0AFDA938448
:100BB000A1829A2031E71385C18FEF0080711375F0
:100BC000F50F9307F03F898F9EA01387C18B930683
:100BD00000F89387C18B74AF74BF2300D702A300C2
:100BE000D7022301D702A301D7021387C7019306B7
:100BF00000062382D7028507E31DF7FEA53D75B7E2
:100C00007D17420741839AA04DF38507A300040096
:100C10001CA061BF1C329386C18BB385D70098217D
:100C20001305B007637DE500850793F7F70F794754
:100C30001CB21D8FE35BF7F689471CA2BDB71107F5
:100C40001377F70F98A1DDDBB387F640F8AF7DB7D8
:100C50001375F50739F9103041C2954763E1C708AC
:100C60001307F6FF931717000967130787683E9766
:100C70001C231833FD177D1793F7F70F1377F70F22
:100C80009545814663E4C500930600F893F5F60F99
:100C900001469386C18B79453308D6002300B800FE
:100CA0000506E31BA6FE794613080006930500041B
:100CB0003385C600230005010506E31BB6FE0DEBD8
:100CC000553B1C301947850793F7F70F1CB0E37E9F
:100CD000F7EC23000400D1BD0147814755B77547A4
:100CE000EDBF3386F60085072300060093F7F70F64
:100CF000E379F7FEF1B7EFF20FC21D891384018289
:100D000029ED1385C18FF123137AF50F9307900F07
:100D100063F5470591450545E92B13791A00B30999
:100D2000240106052380A900AD450545D9239387F5
:100D300041821375F50F3E992300A9001307D00FC8
:100D4000D284637C47019344FAFF83C609008588F7
:100D500033079400BE9414A388A0142091CA9387EB
:100D6000818298232DE303C74182FD1614A098A326
:100D7000183019C7938781829433A1CAFD1694B3A2
:100D80001820930700F8058B11C3814793F6F70FDE
:100D900001479387C18B13064002B305F70094A166
:100DA0000507E31CC7FE143013070006858A91C2AD
:100DB00001479386C7012382E7028507E39DF6FE7C
:100DC00055396FF08FB87D175DB77D1718B003C721
:100DD000518298B375B7EFF2AFB503C7C18293865E
:100DE000018883C8C600EC369387C1822DC37D1766
:100DF00098A390331307400201453306E602938619
:100E0000C18B130340021387C18B1982131805018C
:100E1000135808016315060523001701050505078A
:100E2000E31665FE9C3371477145B387E7020147BE
:100E30009983131607014182639FC7022382160319
:100E400005078506E317A7FE35316FF0AFB098337D
:100E5000D43605071377F70394A398B359BF034813
:100E600007006367B8003308B840230007017DB767
:100E70002300070065B703C646026366B6000D8E01
:100E80002382C60275BF238206025DBFEFF24FAA1E
:100E90001385C18F3D291379F50F1385C18F15294E
:100EA0001374F50F1385C18F2D219307A00F63F6DF
:100EB0002701F9473304F40221809386C18B1387FD
:100EC000C18B01469385C18B1303A00F0D4E930E6A
:100ED0004002130FF0FC130800F8F948637F230366
:100EE00093170601C183631AF4022300E7011DC2B0
:100EF000A30F07FF05060507E31216FF9387C60138
:100F00001307F0032382E6028506E39DD7FE9D3694
:100F10006FF04FA4A3800501F1BF1C236366FE00A0
:100F200085071CA30581F9B763F4FE00FD17D5BF43
:100F3000937F1500E38C0FFEE5B7EFF26F9F938769
:100F40000188C433D4231384C182B9E82310040078
:100F500085441C3013C7170018B013F71700938788
:100F6000C18B31E77946B385E70094A10507E31CFF
:100F7000C7FE13D71600F8AFF8BF2380E702A3809F
:100F8000E7022381E702A381E7021387C7012382D7
:100F9000D7028507E39DE7FEEFF0DFAD04A019A0BF
:100FA0001C20C5DB1C20FD171CA06FF0AF9A014769
:100FB000930640023386E700230006000507E31B83
:100FC000D7FE1387C701238207028507E31DF7FEBB
:100FD000E1B7EFF2EF951387C1821C23BDE31384C1
:100FE000C182138701881430482B782B13F8160020
:100FF00093840188BA8763030800AA8793F5F70FE3
:1010000001469387C18B930840023303F600230007
:10101000B3000506E31B16FF631308002A87137746
:10102000F70F1386C7012382E7028507E39DC7FEFA
:1010300093C6160014B0EFF0FFA3DC381CA06FF0CD
:101040006F91FD171CA3E5BFEFF28F8E1385C18F43
:10105000492401479387C18B930640023306F7006A
:10106000230006000507E31BD7FE1387C701238271
:1010700007028507E31DF7FE23A60182239501825F
:1010800083C7418B194793F7F7F76385E7000D474F
:101090002398E1826FF00F8CEFF28F8903D70183E1
:1010A0008947AA841384018363E2E7081305F00FDC
:1010B000EFF02FA7B7170140114723A8E78021477A
:1010C00023AAE7801E2081E7930790301EA01E20F0
:1010D00013892183FD171EA083A7418313844183B5
:1010E0008DE791650565938505C8130505A0112455
:1010F00008C01385C18FF12A1375F50F9947330581
:10110000F50221812310A90081371C402685FD1797
:101110001CC08357090013972700B7070020938747
:10112000C700BA979C4382976FF0CF82EFF0AFA2CF
:101130009307F00FE31DF5F8B7170140114723AAF5
:10114000E7800145EFF0EF9D59B71387C181230177
:101150000700A3000700238E01808280EFE25FFD7D
:101160001181937715001305E01F91E301459387E3
:10117000E1811387D1819386C1811306F00F930516
:10118000F00FEFF00FDC6FE0FFFCEFE27FFA9387E8
:1011900081838A231307006021054205418133754D
:1011A000E5021387D1819386C1811306F00F930561
:1011B000F00F8AA39387E181EFF0AFD86FE09FF93A
:1011C000EFE21FF71D891384818301ED9307F00B74
:1011D0001385C18F1EA0F5281E200D817D893E95A7
:1011E0000AA010209387E1811387D1819386C18162
:1011F0009305F00F3145EFF0CFD46FE0BFF5EFE28C
:101200003FF31385C18FF1209387818323A00700CB
:1012100023A207006FE01FF4828018414C41104563
:101220000328C5000607B3C7C50005833D8F931685
:10123000170093571800B98EB3C70701B58F1397DE
:10124000A700358F5CC50CC150C118C5858B99C7E7
:101250001C49B18F5CC15C493D8F18C58280EFE2AB
:101260003FEDB717708F9387E71E1CC95CC1B707A6
:1012700079FC9387F7F15CC91CC5B707943793874E
:10128000F7DF3796076C2A840CC11CCD5CC5054777
:101290002145130656966319A700A1442285FD1423
:1012A000AD3FEDFC6FE01FEB9307F7FF8D8B8A07D7
:1012B000A2978C43937637008A0693D7E501AD8FCA
:1012C000B387C702A2968C42BA97AD8F9CC205071E
:1012D000D9B7EFE2FFE52A8489371C441840484417
:1012E000A183BA973D8D858B99C31C4C3D8D6FE0D2
:1012F0007FE6EFE2FFE32A8441111385C18F2EC6FA
:10130000C93FB24542054181818DB385A5024101A6
:10131000C181A2951395050141816FE0BFE3EFE222
:101320003FE137340140AA85854613050480054610
:10133000EF00406913040480C1475CDCA1477CC412
:1013400085452285EF00806689452285EF00807300
:1013500065DDB737014003A5C784420541816FE0D1
:101360007FDF854763ECA700EFE29FDC9387C180B6
:1013700006053E95082165376FE0DFDD41657D1587
:101380008280854763E5A702EFE29FDA1314150018
:101390009387C180A29788235937938701843E940D
:1013A0001E20938717C83325F5006FE0BFDA01458B
:1013B0008280EFE25FD62545056465371304F4FCAF
:1013C00025454537E37EA4FE914401442545FD149F
:1013D000493F93F4F40F2A94F5F885699387F9FF50
:1013E00009807D8C1145239081849389F9FC953F78
:1013F000138901841145B537E3FEA9FE91440144E8
:101400001145FD14B93F93F4F40F2A94F5F84A04FA
:101410005180231189006FE05FD3EFE27FD101118A
:101420001306000281450A85EFE09FD3373401405F
:10143000B7070E003EC68A85854713050480230A38
:10144000F1001123130504808545892B83274480EF
:101450003707000513040480D98F5CC0993F0561EC
:101460006FE05FCF8280EFE2BFCC11C98547630D8B
:10147000F502130700182392E1846FE0BFCD938734
:10148000018883C7470319469386018813F7F70736
:1014900005076373E600014793F707F8D98F238A9E
:1014A000F602EFF07FBAF1B79387018883C757033D
:1014B0000D469386018813F7F70705076373E60067
:1014C000014793F707F8D98FA38AF6020D3B55B76A
:1014D000828037160000B716000037170000938788
:1014E000818593058025130646469386064D13078E
:1014F0006746CCC390C7D4C798CB8CCFD0CF94D3FA
:10150000D8D38280EFE2DFC2938761848823B70655
:1015100000209386C60005051375F50F88A39387F1
:10152000018803C4570383C747039384618493F7F7
:10153000F7078A07B6979C4391C382971374F40701
:10154000B70700209387C7020A043E941C4099C342
:1015500088208297138741841E2381CBFD17C20701
:10156000C1831EA399E3EFF08F94EFE03FF1EFE02A
:101570009FF1AA8513058006EFE01FC96FE09FBDAC
:1015800001A001A0411122C6138781841E23138468
:1015900081848507C207C1831EA31307F03F6379C7
:1015A000F700231004009387C1849843050798C36C
:1015B000EFE0DFDA1E209D8B81CF0547638FE700C8
:1015C0003244B7F700E023A2070041017300203046
:1015D000EFF0AFD3EFF08FCAE5B7EFE09FEECDB7F6
:1015E0008280B707002083A7470681460147A98369
:1015F0001386F7FFB7F700E090CBD4CB814694C7B2
:10160000D8C73D4798C323A207000567B7E700E0A6
:1016100023A0E7108280EFE2BFB1411137140140EF
:101620009307800289443EC64C00930710081305B7
:10163000044026C47C8223130100EF00407493070A
:1016400030224C00130504807C82EF004073930726
:1016500000024C00130504C07C82EF004072B147C9
:1016600041494C00130504807C824AC6EF0020717A
:101670004C00130504802312210102C609274C00E7
:10168000130504C06482E52DE1479304000C4C006F
:10169000130504803EC66482DD2585474C00130592
:1016A00004C07C82E92D91473EC64C00E1771305CA
:1016B00004807C82E925F1474C00130504C03EC636
:1016C0006482752D41016FE0FFA8EFE27FA605451A
:1016D000EF003014192A3705201085450905EF0061
:1016E000902285451305D062EF0010202D37EFF0D2
:1016F0004F92EFE0DFECEFE07FB8EFE05FDBEFF081
:10170000BFB1EFF08FAA0145EFE0BFC1492683D5F5
:10171000618B37F400E0C98D1385C18FEFF03FB4C2
:101720004D3BC135EFF05F92EFF07FAD832704D1E1
:10173000DD9B2328F4D07300501083D781849D8BC8
:10174000F5F7C933E5B7B71702409843B706FFF07E
:101750001367170098C3D843758FD8C39843B7064B
:10176000F7FEFD16758F98C39843B706FCFFFD166C
:10177000758F98C3D843B70601FFFD16758FD8C380
:1017800037079F0098C7B746024003A70680136734
:10179000070123A0E680D843B706C1FFFD16D8C3D2
:1017A000D843D8C3D843D8C3D843758FD8C3D843F8
:1017B000B7061000558FD8C39843B7060001558F60
:1017C00098C3984393166700E3DD06FED843B71627
:1017D0000240719BD8C3D84313672700D8C3214761
:1017E000DC42B18BE39EE7FE8280B7160240DC420A
:1017F0001146B18B138741806385C70021466388FA
:10180000C702B7177A00938707201CC3B717024097
:10181000DC43918393F6F700B70700209387C70353
:10182000B69794231C43B3D7D7001CC38280DC42F5
:10183000D4424166C983BD8BF18E890745466393C7
:10184000C700C94781EEB746024083A60680C18A19
:1018500089CEB7167A009386062021A8B7160240D3
:10186000D4421396E600E35606FEB7163D00938673
:101870000690B387D70251BF01A097F1FF1F938154
:1018800061FE171100201301E1F717150000130581
:10189000A5E097E5FF1F9385E5761386018163FA3E
:1018A000C5008322050023A0550011059105E3EA38
:1018B000C5FE13850181938581916377B50023204F
:1018C00005001105E36DB5FEFD42739002BC8D422B
:1018D00073904280930280087390023097E2FFFF7A
:1018E0009382827293E2320073905230EFF0BFE540
:1018F000970200009382A2DD7390123473002030AF
:10190000EFE21F83B727014093870740631EF5006E
:10191000854513050020EF00F000814513050020E8
:10192000EF0050006FE01F83B737014093870780B7
:10193000E31AF5FE854513050040EF00A07E8145C2
:1019400013050040F1BF5C413707F1E01307F7EFE3
:10195000944D7D8F9C41D58FD44DD58FD441A20617
:10196000D58FD98F5CC11C4537F7F1FF1307D77F9F
:10197000D4457D8F9C49D58F94458606D58FD98FC8
:101980001CC55C55370710FF7D177D8FDC29FD17BF
:1019900093F7F70FD207D98F5CD582801C4589C594
:1019A00093E717001CC58280F99BEDBF1C4591C5CC
:1019B00037075000D98F1CC582803707B0FF7D17CD
:1019C000F98FD5BFA54763F7B7048D47138765FF28
:1019D0003307F7020328C5009D47B397E70093C775
:1019E000F7FFB3F70701B396E600DD8E54C59947BC
:1019F00063E3C70495477D163306F6025859FD4741
:101A0000B397C70093C7F7FFF98F3396C5005D8E74
:101A100050D982800D473387E502032805019D4791
:101A2000B397E70093C7F7FFB3F70701B396E60054
:101A3000DD8E14C96DBFB14763E2C70295476516D5
:101A40003306F6021859FD47B397C70093C7F7FF4F
:101A5000F98F3396C5005D8E10D9828095474D165B
:101A60003306F6025855FD47B397C70093C7F7FFF3
:101A7000F98FB395C500DD8D4CD582806845420550
:101A80004181828008416D8D3335A0008280B7F797
:101A9000FF1F03A5477082800177B706FCFFA1688E
:101AA0000563130E0010B7270240B70E0200370F70
:101AB00004007D17FD166311160503A8070133689E
:101AC000E80123A80701C8CB03A80701136808048D
:101AD00023A8070103A8C70013781800E31C08FE19
:101AE000631A160303A807013378D80023A8070157
:101AF0003295FD15E9F182806317660003A807019E
:101B0000136828007DBFE310C6FD03A807013368F2
:101B1000D80145BF6317660003A807011378D8FFF3
:101B2000F1B7E318C6FD03A80701130505103378C4
:101B3000E80023A8070175BFB70700F8AA97378701
:101B4000030063F3E716EFE20FDD3307B500B78656
:101B50000308AA89AE849307D00F63E9E6123367BE
:101B6000B5001377F70F9307E00F63110712638F28
:101B70000510B7066745B727024093863612379798
:101B8000EFCDD4C31307B79AD8C3D4D3D8D3A167A2
:101B900063E8F5041384F7FFB3758500338AB74013
:101BA0003384F440330945012E946304FA0ED28441
:101BB0006367F404B3078900939A170193DA1A0153
:101BC0004A8B63850A00617B33FB6701B30554418F
:101BD0004A852166BD81C935D28456845A8905A0BB
:101BE000856763E6F5081384F7FFB37585003387CF
:101BF000B7403384F4403309E5002E94BA84056776
:101C000063E2E4029307F7FFB3F7F900014A99C3CF
:101C1000330AF740B38544410566B18133053A0183
:101C2000A53DD284056A63654403B30724017D1A88
:101C300033FA4701CA8A63050A00FD7AB3FA5701ED
:101C4000B30544414A850566B181B9355284568948
:101C500099C41306001093D584004E85353D01CC00
:101C600013060010935584004A853D3529A093073B
:101C7000F00F63E8B702B7270240984BA166558F73
:101C800098CB984B1367070898CB91473E856FE038
:101C9000CFCB2166854509358144E36544F9014A86
:101CA00011BF01440149BDBF9307F00F3E858280FB
:101CB000B70700F8AA973787030063FFE70A3307DF
:101CC000C500B78603089307D00F63E5E60A3367BC
:101CD000C5001377F70F9307E00F49EF41CEB70622
:101CE0006745B7270240938636123797EFCDD4C3A6
:101CF0001307B79AD8C3D4D3C1762182D8D3898D9C
:101D0000C16813030010370E2000FD16984BB38EE8
:101D1000A5003367170198CBD847058B75FFD847C7
:101D2000098B75FF3388EE00032F08003308E500A8
:101D30002320E80103A8C70013782800E31C08FE4D
:101D40001107E31167FE984B130505103367C701B0
:101D500098CBD847058B75FF984B7D16758F98CB20
:101D600055F6984BA166558F98CB984B136707088B
:101D700098CB91473E8582809307F00FE5BF9C4545
:101D800013F7070113F8F70001C7D8413368E800DB
:101D900037270240145B3707000F758F4DEB8546E0
:101DA0002388D184371701406315E5009A213583D4
:101DB0009AA18E2113F7F50F39C318418146854E3C
:101DC0003D4F930F800293028004214E3396DE0034
:101DD000B3F8C500631116039398260033131F014F
:101DE0001343F3FF3377E300B318180133E7E80038
:101DF0006397F70750C98506E39AC6FD18C1130714
:101E0000F00F6375B70454412146854E3D4F930F43
:101E1000800293028004414EB398CE0033F715013F
:101E20006392E8021317260001173313EF001343E0
:101E3000F3FFB376D3003317E800D98E6395F70329
:101E4000232A15010506E319C6FD54C18280371700
:101E50000140E310E5F603C7018521DF81BFE39C64
:101E600057F810C949BFE39F57FC23281501D9BF74
:101E7000EFE20FAC797146212A8468082EC67522DC
:101E8000925737470F001307072433D7E702C204DE
:101E9000C18093F404FCC204B7869303C180938687
:101EA000F66FB24542074183D98C63F4F6001307FD
:101EB000C00346A0162061661306066AC206C182E8
:101EC000F99AC206C18216A094416369D6048606B7
:101ED000B3D7D702114693960701C182B68763F341
:101EE000C6009147C207C1830507420741831AB064
:101EF0005EAC1E20DA21B62593E717001EA01E2037
:101F0000558FC207C18393F757BFD98F1EA09A255B
:101F1000DE25D98F1EA445616FE0CFA3EA2131668B
:101F20007D166319C5020D46B386C602B3D7D70224
:101F3000C207C1839396470199E293E71700A16610
:101F4000D58F9306C0123307D7029306803E3347DE
:101F5000D70259BF6546B386C602B3D7D70291668A
:101F6000C207C183D58FF9B71E2189C593E7170032
:101F70001EA18280C207C183F99BC207C183CDBF66
:101F80001E2189C593E707101EA18280C207C18365
:101F900093F7F7EFC207C183C5BF1E2189C593E739
:101FA00007201EA18280C207C18393F7F7DFC20713
:101FB000C183C5BF0EA9828093F7E50F19C293E7CD
:101FC0001500C207C1831EA982805E290A2D420521
:101FD0005D8D6D8D220521810D8D1335150082805B
:101FE000411102C402C693D7C5012AC63EC4A24706
:101FF000A205A18199CBB247D1073EC6B24788431B
:1020000041016D8D3335A0008280B247C181E10767
:10201000EDB723AAA1848280B7160240DC42517733
:102020007D17F98F5D8DC8C28280371702405C43EF
:102030009146B18B6385D700A1466382D706B71757
:102040007A00938707201CC1371602405C4237078D
:1020500000201307C7049183BD8BBA9794231C41BA
:10206000B3D7D7005CC15442A1829D8ABA9694220C
:10207000B3D6D70014C55442AD829D8A3697182333
:10208000B3D7E7005CC5584239839376370013878E
:10209000818036971823B3D7E7021CC982805C433E
:1020A0005843C166C983BD8B758F8907C546639345
:1020B000D700C94701EF3747024003270780418B0C
:1020C00009CF37177A001307072021A837170240D6
:1020D00058439316E700E3D606FE37173D00130773
:1020E0000790B387E70285B799C5371702401C4FA1
:1020F0005D8D08CF8280B7170240984F1345F5FFDA
:10210000798D88CF828099C5371702405C4F5D8DED
:1021100048CF8280B7170240D84F1345F5FF798D1D
:10212000C8CF828099C5371702405C475D8D48C78C
:102130008280B7170240D8471345F5FF798DC8C78D
:1021400082801E2137370140130707C0C207C183B1
:102150006304E502370700406300E5021307074008
:10216000630CE50037170040930607806306D5002F
:10217000130707C06316E500BA2193F7F7F8D98F64
:10218000FA2193F7F7CFC207C183D98F1EA1DE21B1
:102190005EB59E211EB5B7370140938707C0631413
:1021A000F5009C251EB985475EA982801E319221CB
:1021B00003D82500C207C183F99BC207C1831EB1A2
:1021C0001E3156211A2DC207C1834207418313775E
:1021D000C7F8518F9225F59BC20633660601D18F51
:1021E00037360140130606C0C1826310C502B2250E
:1021F000DD9B03D8E500D18FD221ED9B93F6F6CF7E
:10220000D18FD22533660601D18E56A11AADFA219F
:102210005AB91EB182801E3165771307F7CFC20706
:10222000C183BD9BC207C1831EB11E31562103D895
:102230008500C20713960601162DC18393F7F7FD9B
:10224000758F96214182A206558FB62142074183A0
:10225000B3E606019206D58FB7360140C2079386D2
:1022600006C0C183631ED502B62593F7F7F703D8DE
:10227000C5009206D58FD621C207C183920693F777
:10228000F7FBD58FFD769386F63FF18EF225C207D8
:10229000C183336606010A06D18E13960601418278
:1022A00052A11AADFA211ABD1EB182801E3103D887
:1022B0008500C207C18393F7F7EFC207C1831EB140
:1022C0001E3156215A2DC207139606014207962148
:1022D00041831377C7F8558FB621C18393F7F7DF92
:1022E000B3E60601A206D58FB7360140C207938632
:1022F00006C04182C183631FD502FD769386F67FB7
:10230000F58FB62503D8C500A206D58FD621C20702
:10231000C183A20693F7F7BFD58FF576FD16F18E30
:10232000F225C207C183336606011206D18E1396C9
:102330000601418252A15AADFA215ABD1EB18280D6
:102340001E2189C593E717001EA18280C207C183A1
:10235000F99BC207C183CDBF8357450491C521674F
:10236000D98F2312F5048280C607C583DDBF1E21E5
:1023700089C593E707081EA18280C207C18393F72E
:10238000F7F7C207C183C5BF1E2DC207C183DD9BFE
:10239000DD8D0EAD8280B3C7A5008D8B3307C500E0
:1023A00081E78D4763EDC700AA87637EE508942126
:1023B00085078505A38FD7FEE3EBE7FE8280937642
:1023C0003500AA8789CA942185078505A38FD7FE82
:1023D00093F63700C5BF9376C7FF138606FE63F0FA
:1023E000C70683A3050083A2450083AF850003AF22
:1023F000C50083AE050103AE450103A3850183A893
:10240000C5019385450223A0770003A8C5FF23A239
:10241000570023A4F70123A6E70123A8D70123AA85
:10242000C70123AC670023AE17019387470223AE91
:1024300007FF75B790419107910523AEC7FEE3EB07
:10244000D7FEE3E6E7F682802F2C2A2928262422CD
:10245000201F1E1D1B19151311100F0F0E0E0D0D31
:102460000C0C0C0B0B0B0A0A0A09090908080808CE
:102470000707070707060606FFFFFFFFFFFFFFFF2F
:10248000FF1F1F1F1F1F1F1F000000000100010072
:102490000200020003000300040004000400050021
:1024A00005000600060007000700080008000800F5
:1024B000090009000A000A000B000B000C000C00C8
:1024C0000D000D000E000F000F0010001100110094
:1024D0001200130013001400150016001600170058
:1024E000180019001A001B001C001D001E001F0010
:1024F00020002100220023002400250026002700C0
:1025000028002A002B002C002D002F003000320064
:10251000330034003600370039003A003C003D00FB
:102520003F004100420044004600470049004B0084
:102530004D004F00510053005400560058005A00FF
:102540005D005F0061006300650067006A006C0069
:102550006E0071007300760078007B007D008000C3
:102560008200850088008A008D009000930095000D
:1025700098009B009E00A100A400A700AB00AE0045
:10258000B100B400B700BB00BE00C200C500C80067
:10259000CC00D000D300D700DA00DE00E200E60075
:1025A000EA00ED00F100F500F900FE00020106016D
:1025B0000A010E01130117011B0120012401290149
:1025C0002D01320137013B01400145014A014F0114
:1025D000540159015E01630168016D0172017801C6
:1025E0007D01820188018D01930198019E01A40162
:1025F000A901AF01B501BB01C101C701CD01D301E3
:10260000D901E001E601EC01F301F9010002060243
:102610000D0214021A02210228022F0236023D0284
:1026200044024B02520259026102680270027702B0
:102630007F0286028E0296029D02A502AD02B502BD
:10264000BD02C502CD02D602DE02E602EF02F702AB
:102650000003080311031A0322032B0334033D0371
:1026600046034F03590362036B0375037E0387031D
:1026700091039B03A403AE03B803C203CC03D603A8
:10268000E003EA03F503FF030E150C170918071BF7
:04269000031C000027
:102694000C00000002000000100000003A0F0000CF
:1026A4008C0E0000D60D0000F60C0000D20F0000C6
:1026B400880B000098100000000000004A11000080
:1026C4008A110000C01100005C110000000000002D
:1026D40000000000010203040607080900000000CE
:1026E40001020304010203040607080900000000B4
:1026F40001000000006CDC0202040608090004006A
:00000001FF
